:020000040000FA
:1000000030200020150200001D0200001F02000029
:100010002102000023020000250200000000000071
:1000200000000000000000000000000027020000A7
:1000300029020000000000002B0200002D02000039
:100040005D0200002F0200002F0200002F020000BE
:100050002F0200002F0200002F0200002F020000DC
:100060002F0200002F0200002F020000B502000046
:100070002F0200002F0200002F0200002F020000BC
:100080002F0200002F0200002F0200002F020000AC
:100090002F0200002F0200002F0200002F0200009C
:1000A0002F0200002F0200002F0200002F0200008C
:1000B0002F0200002F0200000000000000000000DE
:1000C0002F0200002F0200002F0200002F0200006C
:1000D0002F0200002F0200002F020000000000008D
:1000E0000000000000000000000000000000000010
:1000F0000000000000000000000000000000000000
:1001000000000000000000000000000000000000EF
:1001100000000000000000000000000000000000DF
:1001200000000000000000000000000000000000CF
:1001300000000000000000000000000000000000BF
:1001400000000000000000000000000000000000AF
:10015000000000000000000000000000000000009F
:10016000000000000000000000000000000000008F
:10017000000000000000000000000000000000007F
:10018000000000000000000000000000000000006F
:10019000000000000000000000000000000000005F
:1001A000000000000000000000000000000000004F
:1001B000000000000000000000000000000000003F
:1001C000000000000000000000000000000000002F
:1001D000000000000000000000000000000000001F
:1001E000000000000000000000000000000000000F
:1001F00000000000000000000000000000000000FF
:10020000DFF80CD000F018F800480047E9070000BC
:10021000302000200648804706480047FEE7FEE7FA
:10022000FEE7FEE7FEE7FEE7FEE7FEE7FEE7FEE7A6
:10023000C502000001020000064C074D06E0E06820
:1002400040F0010394E8070098471034AC42F6D31D
:10025000FFF7DAFF6C0B00008C0B000070B54FF459
:100260008076304600F0FAFA114CB50560B13046A0
:1002700000F0FBFA0120C5F80803607920B90120DD
:1002800060712168002088474FF48276304600F084
:10029000E5FA00280AD0304600F0E7FA0220C5F857
:1002A00008032168BDE870400120084770BD0000C8
:1002B0000000002003220021014800F039BA0000AC
:1002C00000B00040F0B5B5480023021D0178101DB4
:1002D00001254FF0805406290BD11678360708D136
:1002E0000678C6F30316032E06D0042E04D0052E7E
:1002F00002D0062907D00EE0B4F82463A84FC6F355
:1003000004263E6002E01678360704D10678C6F36C
:100310000316032E02D0062904D00FE0A24FA14EEF
:100320007E670EE01678360708D10678C6F3031606
:10033000032E06D0042E04D0052E02D0062907D0A5
:100340000EE0D4F84462994FC6F342363E6002E0B4
:100350001678360704D10678C6F30316032E02D0AA
:10036000062906D011E0924E376827F08077376073
:100370000EE01678360708D10678C6F30316032E6A
:1003800006D0042E04D0052E02D006290AD011E092
:100390004FF08046C6F80C31C6F81031834E361F38
:1003A000336002E01678360704D10678C6F30316E8
:1003B000032E02D0062905D00CE07C4F03266437BB
:1003C0003E600AE01678360704D10678C6F30316B5
:1003D000032E02D006290DD014E0764F05263E608C
:1003E000744E78363560734E083633603F263F1DB5
:1003F0003E6002E01678360704D10678C6F303168D
:10040000052E02D0062957D062E06B4E36686B4F3E
:100410003E60694E361D36683F1D3E60664E0836AA
:1004200036683F1D3E60644E0C3636683F1D3E60A8
:10043000614E103636683F1D3E605F4E143636689A
:100440003F1D3E605C4E183636685C4F20373E607C
:10045000594E1C3636683F1D3E60574E2036366872
:100460003F1D3E60544E243636683F1D3E60524E5E
:10047000283636683F1D3E604F4E2C3636683F1D8D
:100480003E604D4E303636684C4F40373E604A4EE7
:10049000343636683F1D3E60474E383636683F1D5D
:1004A0003E60454E3C3636683F1D3E60424E40360B
:1004B00036683F1D3E6002E01678360708D10678A0
:1004C000C6F30316032E06D0042E04D0052E02D048
:1004D000062907D019E0D4F85812394A01F04F0123
:1004E000116002E0117809070FD10078C0F3031002
:1004F000032803D0042801D0052806D1314801681B
:10050000C90702D06FF001010160D4F8300106285C
:1005100008D1D4F83401062804D12B48016841F4ED
:100520008061016022487438016841F47001016003
:10053000BFF34F8FBFF36F8F4FF01021D1F8000240
:10054000002803DBD1F80402002822DA1F4A1560D4
:100550001F480468002CFCD01524C1F8004205682F
:10056000002DFCD0C1F8044201680029FCD01360C2
:1005700001680029FCD0BFF34F8F0D48F0380168A7
:10058000144A01F4E06111430160BFF34F8F00BFD3
:10059000FDE7124910480860F0BD0000E00F00F0D0
:1005A000403501400DF0ADBA00C007403C050040A9
:1005B000FCED00E0105600400404001020C500408F
:1005C000E40E0040000400403C17004004E50140F8
:1005D00000E401400400FA050090D003140000205C
:1005E00002E008C8121F08C1002AFAD170477047FC
:1005F000002001E001C1121F002AFBD1704700005A
:1006000072B609480068C00700D000BEBFF34F8F24
:100610000548E4380168054A01F4E06111430160CE
:10062000BFF34F8F00BFFDE7F0ED00E00400FA05D7
:100630000EB500210091CDE901106A4644F2010097
:10064000FFF7DEFF0EBD00F003B800F009B80000B0
:1006500072B602480168491C016070471000002012
:1006600003490868401E086000D162B67047000068
:10067000100000202DE9FC410646C0074FF00005A0
:100680000ED0104F00240122385D00950023114642
:10069000019500F031F9641C042CF4D300F01CF82F
:1006A000B0070DD5074E0024361D0022305D032310
:1006B00000951146019500F01FF9641C042CF4D339
:1006C000BDE8FC81640B00000249085C012100F0D8
:1006D00033B90000640B000010B500242046FFF77A
:1006E000F3FF641C042CF9D310BD000070B5084C56
:1006F000050009D010342168002907D0086820605F
:10070000496828468847F6E70834F4E770BD0000DA
:1007100018000020054A012120B1012805D191705F
:10072000FFF7E4BF51700020FAE77047180000207F
:100730002DE9F0479146884604464FF480354FF442
:10074000A0760027DFF884A016E000BFD4F80403E9
:1007500028420DD0A05958B1C4F84853C4F80853E2
:100760003146204600F0F3F85AF82810F8B28847CE
:10077000361D6D00B6B27F1C4F45E7D3D4F8040395
:100780004FF4807110F0010F09D0D4F8000130B19E
:10079000204600F0DCF85AF8281004208847D4F8E6
:1007A00004034FF4827110F0020F0CD0D4F804014E
:1007B000002808D0204600F0CAF85AF82810BDE8F2
:1007C000F04705200847BDE8F08700000C00002036
:1007D0000268134602E08A4204D01268002AFAD165
:1007E0000B600160704700001CB50120FFF742FF5D
:1007F00000F044F808B1FFF71BFF002000F058F8A4
:100800001449154AD1E90001CDE9000140F6FF7015
:10081000ADF800000F486946083000F039F908B11A
:10082000FFF706FF0B480121083000F077F909486F
:10083000012318220021083000F0DCF808B1FFF78E
:10084000F7FE0448083000F017F940BF20BF20BF72
:10085000FBE70000540B0000410B000000F180405A
:100860000068002800D00120704708B500F18040E2
:10087000002101600068009008BD000070B50A4CBE
:10088000207808B185250CE00020A0606060206120
:10089000E060064800F078F8054600F05FF80120B7
:1008A0002070284670BD00001800002015070000C9
:1008B00070B5104D0446A87838B114B161680120B4
:1008C00088470020FFF7BFFE0CE00020FFF7BBFECB
:1008D00024B1084821461030FFF77AFFE86808B9CC
:1008E00000F062F8E868401CE860BDE87040002055
:1008F000FFF7ABBE1800002070B541EA4201DDE908
:1009000004564FF0A04441EA830141EA052104EB7B
:10091000800041EA0641C0F8001770BD4FF0A042C8
:10092000D2F804350121814021EA0300C2F808050C
:100930001940C2F80C15704701224FF0A0438240C5
:1009400011B1C3F808257047C3F80C25704708B5E6
:10095000002242504058009008BD0000084800683E
:10096000012110F0010F08D14FF0E020E02280F8C3
:100970000024C0F88012C0F80011024801607047DE
:1009800000E100E0180500400649024600200B790E
:100990000BB1852070470A6001220A7100224A715A
:1009A000704700000000002070B54FF48270FFF720
:1009B0005CFF02204107C1F804030B4B196841F0AA
:1009C000807018600948026842F0010404604468BD
:1009D0004FF40A554668361BAE42FBD302601960DD
:1009E00003490120086070BDFCED00E0001000E04C
:1009F000080000402DE9F04105464FF4A07000EBDF
:100A0000810086B228684FF480348C40C0F8484397
:100A10002868C0F8084322F07F406A79154F02EB3E
:100A200042023A445278002A2A6802EB8101C1F856
:100A3000400512D02968D1F80425111A824202D249
:100A40006FF07F400144687900EB400038448078C3
:100A5000884202DD0D20BDE8F08133B131462868BF
:100A6000FFF775FF2868C0F804432868C0F84443BE
:100A70000020F0E708000020016801220A604079A8
:100A8000024A00EB40000221115470470800002088
:100A900070B54379204C44F823204279231F02EBA0
:100AA00042029A5C0AB1082070BD90F904208C784B
:100AB000002A4FEA441406DA02F00F0202F1E022A3
:100AC00082F8144D03E002F1E02282F8004490F92C
:100AD0000420012502F01F0605FA06F452099200CF
:100AE00002F1E022C2F88042C2F8004102680C889C
:100AF000C2F8084544790A7904EB44041C44627046
:100B00004279C97802EB42021A449170407900EBB5
:100B100040001D54002070BD0C00002070B50E4632
:100B200005464FF4807101240068FFF710FF286824
:100B3000C0F84443002E02D02868C0F8044370BDBA
:100B400020B1042804D11120FFF7E8BE1220FBE7F2
:100B500070470000000007410000000000B00040A6
:100B60000B000300111213140D0E0F108C0B00005C
:100B70000000002018000000E0050000A40B0000A9
:100B80001800002018200000F00500000000000000
:100B90000000000000000000000000000000000055
:040BA0000090D003EE
:0400000500000201F4
:00000001FF
